000: 01 11     IRQ0 Vector 0111h
002: 88 58     IRQ1 Vector 8858h
004: 00 00     IRQ2 Vector 0000h
006: 00 00     IRQ3 Vector 0000h
008: 00 00     IRQ4 Vector 0000h
00a: 01 5c     IRQ5 Vector 015Ch
00c: 31 f0     SRP  #F0h
00e: 8c 4d     LD   R8, #4Dh
010: 7c 00     LD   R7, #00h
012: 6c 00     LD   R6, #00h
014: bc 20     LD   R11, #20h
016: 2c fa     LD   R2, #FAh
018: 3c a3     LD   R3, #A3h
01a: 1c 0c     LD   R1, #0Ch
01c: 31 10     SRP  #10h
01e: e6 03 00  LD   P3, #00h
021: e6 ff 80  LD   SPL, #80h
024: e6 0f c8  LD   0Fh, #C8h
027: d6 03 37  CALL 0337h
02a: e6 04 05  LD   04h, #05h
02d: a6 04 05  CP   04h, #05h
030: ed 00 a4  JP   NZ, 00A4h
033: e7 04 55  LD   @04h, #55h
036: a7 04 55  CP   @04h, #55h
039: ed 00 a4  JP   NZ, 00A4h
03c: e7 04 aa  LD   @04h, #AAh
03f: a7 04 aa  CP   @04h, #AAh
042: ed 00 a4  JP   NZ, 00A4h
045: b1 04     CLR  @04h
047: a7 04 00  CP   @04h, #00h
04a: ed 00 a4  JP   NZ, 00A4h
04d: 20 04     INC  04h
04f: a6 04 80  CP   04h, #80h
052: 1b df     JR   LT, 0033h
054: b0 0d     CLR  0Dh
056: b0 0e     CLR  0Eh
058: b0 04     CLR  04h
05a: e6 07 0a  LD   07h, #0Ah
05d: e6 06 32  LD   06h, #32h
060: e6 31 20  LD   31h, #20h
063: 76 03 02  TM   P3, #02h
066: eb b6     JR   NZ, 001Eh
068: e6 0f 37  LD   0Fh, #37h
06b: d6 03 37  CALL 0337h
06e: 0c 52     LD   R0, #52h
070: 1c 10     LD   R1, #10h
072: d6 02 f7  CALL 02F7h
075: fc aa     LD   R15, #AAh
077: d6 02 5d  CALL 025Dh
07a: 9f        EI   
07b: b0 0c     CLR  0Ch
07d: 7c 32     LD   R7, #32h
07f: e6 62 fe  LD   62h, #FEh
082: e4 62 02  LD   P2, 62h
085: 0c 0c     LD   R0, #0Ch
087: 0a fe     DJNZ R0, 0087h
089: f5 00 e7  LD   @00h, R7
08c: 61 e7     COM  @R7
08e: 7e        INC  R7
08f: f5 01 e7  LD   @01h, R7
092: 61 e7     COM  @R7
094: 7e        INC  R7
095: a6 e7 42  CP   R7, #42h
098: 6b 16     JR   Z, 00B0h
09a: 90 62     RL   62h
09c: e4 62 02  LD   P2, 62h
09f: d6 02 73  CALL 0273h
0a2: 8b e1     JR   0085h
0a4: fc fc     LD   R15, #FCh
0a6: d6 02 94  CALL 0294h
0a9: eb f9     JR   NZ, 00A4h
0ab: d6 02 f0  CALL 02F0h
0ae: 8b fb     JR   00ABh
0b0: a6 0c 00  CP   0Ch, #00h
0b3: eb 0b     JR   NZ, 00C0h
0b5: dc 32     LD   R13, #32h
0b7: ec 42     LD   R14, #42h
0b9: d6 03 01  CALL 0301h
0bc: 20 0c     INC  0Ch
0be: 8b bd     JR   007Dh
0c0: dc 32     LD   R13, #32h
0c2: ec 42     LD   R14, #42h
0c4: d6 03 0e  CALL 030Eh
0c7: eb b2     JR   NZ, 007Bh
0c9: a6 0c 0f  CP   0Ch, #0Fh
0cc: eb ee     JR   NZ, 00BCh
0ce: d6 03 1d  CALL 031Dh
0d1: a6 e1 03  CP   R1, #03h
0d4: ab a5     JR   GT, 007Bh
0d6: dc 42     LD   R13, #42h
0d8: ec 52     LD   R14, #52h
0da: b0 ec     CLR  R12
0dc: e5 ed 0b  LD   0Bh, @R13
0df: b5 ee 0b  XOR  0Bh, @R14
0e2: eb 36     JR   NZ, 011Ah
0e4: de        INC  R13
0e5: ee        INC  R14
0e6: ce        INC  R12
0e7: a6 ec 10  CP   R12, #10h
0ea: eb f0     JR   NZ, 00DCh
0ec: a6 04 00  CP   04h, #00h
0ef: 6b 1f     JR   Z, 0110h
0f1: a6 04 03  CP   04h, #03h
0f4: eb 05     JR   NZ, 00FBh
0f6: a6 05 6a  CP   05h, #6Ah
0f9: 6b 15     JR   Z, 0110h
0fb: a4 06 09  CP   09h, 06h
0fe: eb 10     JR   NZ, 0110h
100: a4 07 08  CP   08h, 07h
103: eb 0b     JR   NZ, 0110h
105: 88 04     LD   R8, 04h
107: 98 05     LD   R9, 05h
109: 6c 00     LD   R6, #00h
10b: d6 01 8b  CALL 018Bh
10e: b0 08     CLR  08h
110: dc 42     LD   R13, #42h
112: ec 52     LD   R14, #52h
114: d6 03 01  CALL 0301h
117: 8d 00 7b  JP   007Bh
11a: b8 0b     LD   R11, 0Bh
11c: 53 bd     AND  R11, @R13
11e: ac ff     LD   R10, #FFh
120: d6 01 6b  CALL 016Bh
123: a6 ea 08  CP   R10, #08h
126: 6b 10     JR   Z, 0138h
128: d6 01 76  CALL 0176h
12b: 89 04     LD   04h, R8
12d: 98 05     LD   R9, 05h
12f: 6c 00     LD   R6, #00h
131: d6 01 8b  CALL 018Bh
134: b0 09     CLR  09h
136: 8b e8     JR   0120h
138: b8 0b     LD   R11, 0Bh
13a: 53 be     AND  R11, @R14
13c: ac ff     LD   R10, #FFh
13e: d6 01 6b  CALL 016Bh
141: a6 ea 08  CP   R10, #08h
144: 6b 9e     JR   Z, 00E4h
146: d6 01 76  CALL 0176h
149: a4 e8 04  CP   04h, R8
14c: eb 07     JR   NZ, 0155h
14e: a4 e9 05  CP   05h, R9
151: eb 02     JR   NZ, 0155h
153: b0 04     CLR  04h
155: 6c 80     LD   R6, #80h
157: d6 01 8b  CALL 018Bh
15a: 8b e2     JR   013Eh
15c: a4 06 09  CP   09h, 06h
15f: 6b 02     JR   Z, 0163h
161: 20 09     INC  09h
163: a4 07 08  CP   08h, 07h
166: 6b 02     JR   Z, 016Ah
168: 20 08     INC  08h
16a: bf        IRET 
16b: ae        INC  R10
16c: e0 eb     RR   R11
16e: 7b 05     JR   C, 0175h
170: a6 ea 08  CP   R10, #08h
173: eb f6     JR   NZ, 016Bh
175: af        RET  
176: 98 ec     LD   R9, R12
178: 90 e9     RL   R9
17a: 90 e9     RL   R9
17c: 90 e9     RL   R9
17e: 02 9a     ADD  R9, R10
180: 90 e9     RL   R9
182: 06 e9 4e  ADD  R9, #4Eh
185: 8c 03     LD   R8, #03h
187: 16 e8 00  ADC  R8, #00h
18a: af        RET  
18b: a6 e8 03  CP   R8, #03h
18e: eb 0d     JR   NZ, 019Dh
190: a6 e9 5a  CP   R9, #5Ah
193: eb 08     JR   NZ, 019Dh
195: b0 0e     CLR  0Eh
197: 42 66     OR   R6, R6
199: eb 02     JR   NZ, 019Dh
19b: 20 0e     INC  0Eh
19d: a6 e8 03  CP   R8, #03h
1a0: eb 15     JR   NZ, 01B7h
1a2: a6 e9 6a  CP   R9, #6Ah
1a5: eb 10     JR   NZ, 01B7h
1a7: 42 66     OR   R6, R6
1a9: 6b 01     JR   Z, 01ACh
1ab: af        RET  
1ac: 44 0e 0e  OR   0Eh, 0Eh
1af: 6b 73     JR   Z, 0224h
1b1: 8c 04     LD   R8, #04h
1b3: 9c 58     LD   R9, #58h
1b5: 8b 6d     JR   0224h
1b7: 44 0e 0e  OR   0Eh, 0Eh
1ba: ed 02 24  JP   NZ, 0224h
1bd: a6 e8 03  CP   R8, #03h
1c0: eb 1e     JR   NZ, 01E0h
1c2: a6 e9 ec  CP   R9, #ECh
1c5: eb 19     JR   NZ, 01E0h
1c7: 42 62     OR   R6, R2
1c9: 6b 05     JR   Z, 01D0h
1cb: 56 0d f7  AND  0Dh, #F7h
1ce: 8b 54     JR   0224h
1d0: 76 0d 08  TM   0Dh, #08h
1d3: eb 4f     JR   NZ, 0224h
1d5: 42 0d     OR   R0, R13
1d7: 08 b6     LD   R0, B6h
1d9: 0f        Illegal
1da: 08 d6     LD   R0, D6h
1dc: 03 37     ADD  R3, @R7
1de: 8b 44     JR   0224h
1e0: a6 e8 03  CP   R8, #03h
1e3: eb 1e     JR   NZ, 0203h
1e5: a6 e9 9a  CP   R9, #9Ah
1e8: eb 19     JR   NZ, 0203h
1ea: 42 66     OR   R6, R6
1ec: 6b 05     JR   Z, 01F3h
1ee: 56 0d 7f  AND  0Dh, #7Fh
1f1: 8b 31     JR   0224h
1f3: 76 0d 80  TM   0Dh, #80h
1f6: eb 2c     JR   NZ, 0224h
1f8: 46 0d 80  OR   0Dh, #80h
1fb: b6 0f 80  XOR  0Fh, #80h
1fe: d6 03 37  CALL 0337h
201: 8b 21     JR   0224h
203: a6 e8 03  CP   R8, #03h
206: eb 1c     JR   NZ, 0224h
208: a6 e9 e2  CP   R9, #E2h
20b: eb 17     JR   NZ, 0224h
20d: 42 66     OR   R6, R6
20f: 6b 05     JR   Z, 0216h
211: 56 0d bf  AND  0Dh, #BFh
214: 8b 0e     JR   0224h
216: 76 0d 40  TM   0Dh, #40h
219: eb 09     JR   NZ, 0224h
21b: 46 0d 40  OR   0Dh, #40h
21e: b6 0f 40  XOR  0Fh, #40h
221: d6 03 37  CALL 0337h
224: c2 f8     LDC  R15, @RR8
226: 76 ef 08  TM   R15, #08h
229: eb 14     JR   NZ, 023Fh
22b: 76 ef 01  TM   R15, #01h
22e: 6b 05     JR   Z, 0235h
230: fc e0     LD   R15, #E0h
232: d6 02 5d  CALL 025Dh
235: a0 e8     INCW R8
237: c2 f8     LDC  R15, @RR8
239: 42 f6     OR   R15, R6
23b: d6 02 5d  CALL 025Dh
23e: af        RET  
23f: 56 ef f0  AND  R15, #F0h
242: f0 ef     SWAP R15
244: 78 ef     LD   R7, R15
246: c2 f8     LDC  R15, @RR8
248: 56 ef 07  AND  R15, #07h
24b: a0 e8     INCW R8
24d: c2 98     LDC  R9, @RR8
24f: 88 ef     LD   R8, R15
251: c2 f8     LDC  R15, @RR8
253: 42 f6     OR   R15, R6
255: d6 02 5d  CALL 025Dh
258: a0 e8     INCW R8
25a: 7a f5     DJNZ R7, 0251h
25c: af        RET  
25d: a6 31 31  CP   31h, #31h
260: 6b 10     JR   Z, 0272h
262: a6 31 30  CP   31h, #30h
265: eb 06     JR   NZ, 026Dh
267: e7 31 ff  LD   @31h, #FFh
26a: 20 31     INC  31h
26c: af        RET  
26d: f5 ef 31  LD   @R15, 31h
270: 20 31     INC  31h
272: af        RET  
273: d6 02 f0  CALL 02F0h
276: a6 31 20  CP   31h, #20h
279: 6b 07     JR   Z, 0282h
27b: f8 20     LD   R15, 20h
27d: d6 02 94  CALL 0294h
280: 6b 01     JR   Z, 0283h
282: af        RET  
283: 0c 10     LD   R0, #10h
285: 1c 21     LD   R1, #21h
287: 2c 20     LD   R2, #20h
289: e3 31     LD   R3, @R1
28b: f3 23     LD   @R2, R3
28d: 1e        INC  R1
28e: 2e        INC  R2
28f: 0a f8     DJNZ R0, 0289h
291: 00 31     DEC  31h
293: af        RET  
294: d6 02 f0  CALL 02F0h
297: e6 03 c0  LD   P3, #C0h
29a: 70 e1     PUSH R1
29c: 50 e1     POP  R1
29e: 1c 0f     LD   R1, #0Fh
2a0: e6 03 40  LD   P3, #40h
2a3: 76 03 01  TM   P3, #01h
2a6: 6b 07     JR   Z, 02AFh
2a8: 1a f9     DJNZ R1, 02A3h
2aa: e6 03 80  LD   P3, #80h
2ad: 1e        INC  R1
2ae: af        RET  
2af: f9 0a     LD   0Ah, R15
2b1: 2c 28     LD   R2, #28h
2b3: d6 02 fe  CALL 02FEh
2b6: e6 03 40  LD   P3, #40h
2b9: d6 02 d9  CALL 02D9h
2bc: 60 ef     COM  R15
2be: 1c 08     LD   R1, #08h
2c0: e0 ef     RR   R15
2c2: 08 ef     LD   R0, R15
2c4: 46 e0 40  OR   R0, #40h
2c7: 09 03     LD   P3, R0
2c9: d6 02 d9  CALL 02D9h
2cc: 1a f2     DJNZ R1, 02C0h
2ce: 2c 03     LD   R2, #03h
2d0: d6 02 fe  CALL 02FEh
2d3: e6 03 80  LD   P3, #80h
2d6: b2 11     XOR  R1, R1
2d8: af        RET  
2d9: e4 10 10  LD   10h, 10h
2dc: 56 03 80  AND  P3, #80h
2df: d6 02 f0  CALL 02F0h
2e2: 2c 14     LD   R2, #14h
2e4: d6 02 fe  CALL 02FEh
2e7: 46 03 40  OR   P3, #40h
2ea: 2c 04     LD   R2, #04h
2ec: d6 02 fe  CALL 02FEh
2ef: af        RET  
2f0: 76 03 02  TM   P3, #02h
2f3: ed 00 1e  JP   NZ, 001Eh
2f6: af        RET  
2f7: e7 e0 00  LD   @R0, #00h
2fa: 0e        INC  R0
2fb: 1a fa     DJNZ R1, 02F7h
2fd: af        RET  
2fe: 2a fe     DJNZ R2, 02FEh
300: af        RET  
301: 18 ee     LD   R1, R14
303: e3 0d     LD   R0, @R13
305: f3 e0     LD   @R14, R0
307: de        INC  R13
308: ee        INC  R14
309: a2 d1     CP   R13, R1
30b: eb f6     JR   NZ, 0303h
30d: af        RET  
30e: 18 ee     LD   R1, R14
310: e3 0e     LD   R0, @R14
312: a3 0d     CP   R0, @R13
314: eb 06     JR   NZ, 031Ch
316: ee        INC  R14
317: de        INC  R13
318: a2 d1     CP   R13, R1
31a: eb f4     JR   NZ, 0310h
31c: af        RET  
31d: 0c 42     LD   R0, #42h
31f: b0 e1     CLR  R1
321: e3 b0     LD   R11, @R0
323: ac ff     LD   R10, #FFh
325: d6 01 6b  CALL 016Bh
328: a6 ea 08  CP   R10, #08h
32b: 6b 03     JR   Z, 0330h
32d: 1e        INC  R1
32e: 8b f5     JR   0325h
330: 0e        INC  R0
331: a6 e0 52  CP   R0, #52h
334: eb eb     JR   NZ, 0321h
336: af        RET  
337: 0c 08     LD   R0, #08h
339: 46 03 20  OR   P3, #20h
33c: 46 03 10  OR   P3, #10h
33f: 90 0f     RL   0Fh
341: fb 03     JR   NC, 0346h
343: 56 03 ef  AND  P3, #EFh
346: d2 20     LDC  @RR0, R2
348: 0a f2     DJNZ R0, 033Ch
34a: 56 03 df  AND  P3, #DFh
34d: af        RET  
34e: 00 02     DEC  P2
350: 00 04     DEC  04h
352: 00 06     DEC  06h
354: 00 08     DEC  08h
356: 00 0a     DEC  0Ah
358: 00 0c     DEC  0Ch
35a: 00 1d     DEC  1Dh
35c: 00 4a     DEC  4Ah
35e: 01 4d     DEC  @4Dh
360: 01 52     DEC  @52h
362: 01 49     DEC  @49h
364: 01 35     DEC  @35h
366: 00 00     DEC  P0
368: 00 00     DEC  P0
36a: 6c 4e     LD   R6, #4Eh
36c: 00 00     DEC  P0
36e: 00 10     DEC  10h
370: 00 12     DEC  12h
372: 00 14     DEC  14h
374: 00 16     DEC  16h
376: 00 18     DEC  18h
378: 00 1a     DEC  1Ah
37a: 00 36     DEC  36h
37c: 00 00     DEC  P0
37e: 01 50     DEC  @50h
380: 01 53     DEC  @53h
382: 01 51     DEC  @51h
384: 00 48     DEC  48h
386: 00 00     DEC  P0
388: 00 00     DEC  P0
38a: 00 57     DEC  57h
38c: 00 58     DEC  58h
38e: 00 1e     DEC  1Eh
390: 00 20     DEC  20h
392: 00 22     DEC  22h
394: 00 24     DEC  24h
396: 00 26     DEC  26h
398: 00 28     DEC  28h
39a: 00 3a     DEC  3Ah
39c: 00 4e     DEC  4Eh
39e: 01 4b     DEC  @4Bh
3a0: 00 00     DEC  P0
3a2: 00 00     DEC  P0
3a4: 00 4c     DEC  4Ch
3a6: 00 00     DEC  P0
3a8: 00 00     DEC  P0
3aa: 00 42     DEC  42h
3ac: 00 00     DEC  P0
3ae: 00 2c     DEC  2Ch
3b0: 00 2e     DEC  2Eh
3b2: 00 30     DEC  30h
3b4: 00 32     DEC  32h
3b6: 00 34     DEC  34h
3b8: 00 00     DEC  P0
3ba: 00 2a     DEC  2Ah
3bc: 01 1c     DEC  @1Ch
3be: 00 1c     DEC  1Ch
3c0: 00 00     DEC  P0
3c2: 00 00     DEC  P0
3c4: 00 50     DEC  50h
3c6: 00 00     DEC  P0
3c8: 00 00     DEC  P0
3ca: 00 3e     DEC  3Eh
3cc: 00 3f     DEC  3Fh
3ce: 00 03     DEC  P3
3d0: 00 05     DEC  05h
3d2: 00 07     DEC  07h
3d4: 00 09     DEC  09h
3d6: 00 0b     DEC  0Bh
3d8: 00 0d     DEC  0Dh
3da: 00 56     DEC  56h
3dc: 00 0e     DEC  0Eh
3de: 00 52     DEC  52h
3e0: 01 47     DEC  @47h
3e2: 00 45     DEC  45h
3e4: 00 37     DEC  37h
3e6: 00 49     DEC  49h
3e8: 00 00     DEC  P0
3ea: 01 37     DEC  @37h
3ec: 00 46     DEC  46h
3ee: 00 11     DEC  11h
3f0: 00 13     DEC  13h
3f2: 00 15     DEC  15h
3f4: 00 17     DEC  17h
3f6: 00 19     DEC  19h
3f8: 00 1b     DEC  1Bh
3fa: 00 01     DEC  P1
3fc: 00 0f     DEC  0Fh
3fe: 4c 5a     LD   R4, #5Ah
400: 01 4f     DEC  @4Fh
402: 00 47     DEC  47h
404: 00 49     DEC  49h
406: 00 3b     DEC  3Bh
408: 00 00     DEC  P0
40a: 00 43     DEC  43h
40c: 00 44     DEC  44h
40e: 00 1f     DEC  1Fh
410: 00 21     DEC  21h
412: 00 23     DEC  23h
414: 00 25     DEC  25h
416: 00 27     DEC  27h
418: 00 2b     DEC  2Bh
41a: 00 36     DEC  36h
41c: 00 29     DEC  29h
41e: 00 53     DEC  53h
420: 00 00     DEC  P0
422: 00 4b     DEC  4Bh
424: 00 4d     DEC  4Dh
426: 00 00     DEC  P0
428: 00 38     DEC  38h
42a: 00 40     DEC  40h
42c: 00 41     DEC  41h
42e: 00 2d     DEC  2Dh
430: 00 2f     DEC  2Fh
432: 00 31     DEC  31h
434: 00 33     DEC  33h
436: 00 35     DEC  35h
438: 00 00     DEC  P0
43a: 00 00     DEC  P0
43c: 00 39     DEC  39h
43e: 00 00     DEC  P0
440: 01 48     DEC  @48h
442: 00 4f     DEC  4Fh
444: 00 51     DEC  51h
446: 00 54     DEC  54h
448: 01 38     DEC  @38h
44a: 00 3c     DEC  3Ch
44c: 00 3d     DEC  3Dh
44e: e1 1d     RR   @1Dh
450: 45 e1 9d  OR   9Dh, @R1
453: c5        Illegal
454: e0 46     RR   46h
456: e0 c6     RR   C6h
458: 4c 54     LD   R4, #54h
45a: e1 52     RR   @52h
45c: e1 52     RR   @52h
45e: ff        NOP  
45f: ff        NOP  
460: ff        NOP  
461: ff        NOP  
462: ff        NOP  
463: ff        NOP  
464: ff        NOP  
465: ff        NOP  
466: ff        NOP  
467: ff        NOP  
468: ff        NOP  
469: ff        NOP  
46a: ff        NOP  
46b: ff        NOP  
46c: ff        NOP  
46d: ff        NOP  
46e: ff        NOP  
46f: ff        NOP  
470: ff        NOP  
471: ff        NOP  
472: ff        NOP  
473: ff        NOP  
474: ff        NOP  
475: ff        NOP  
476: ff        NOP  
477: ff        NOP  
478: ff        NOP  
479: ff        NOP  
47a: ff        NOP  
47b: ff        NOP  
47c: ff        NOP  
47d: ff        NOP  
47e: ff        NOP  
47f: ff        NOP  
480: 00 00     DEC  P0
482: 00 00     DEC  P0
484: 00 00     DEC  P0
486: 00 00     DEC  P0
488: 00 00     DEC  P0
48a: 00 00     DEC  P0
48c: 00 00     DEC  P0
48e: 00 00     DEC  P0
490: 00 00     DEC  P0
492: 00 00     DEC  P0
494: 00 00     DEC  P0
496: 00 00     DEC  P0
498: 00 00     DEC  P0
49a: 00 00     DEC  P0
49c: 00 00     DEC  P0
49e: 00 00     DEC  P0
4a0: 00 00     DEC  P0
4a2: 00 00     DEC  P0
4a4: 00 00     DEC  P0
4a6: 00 00     DEC  P0
4a8: 00 00     DEC  P0
4aa: 00 00     DEC  P0
4ac: 00 00     DEC  P0
4ae: 00 00     DEC  P0
4b0: 00 00     DEC  P0
4b2: 00 00     DEC  P0
4b4: 00 00     DEC  P0
4b6: 00 00     DEC  P0
4b8: 00 00     DEC  P0
4ba: 00 00     DEC  P0
4bc: 00 00     DEC  P0
4be: 00 00     DEC  P0
4c0: 00 00     DEC  P0
4c2: 00 00     DEC  P0
4c4: 00 00     DEC  P0
4c6: 00 00     DEC  P0
4c8: 00 00     DEC  P0
4ca: 00 00     DEC  P0
4cc: 00 00     DEC  P0
4ce: 00 00     DEC  P0
4d0: 00 00     DEC  P0
4d2: 00 00     DEC  P0
4d4: 00 00     DEC  P0
4d6: 00 00     DEC  P0
4d8: 00 00     DEC  P0
4da: 00 00     DEC  P0
4dc: 00 00     DEC  P0
4de: 00 00     DEC  P0
4e0: 00 00     DEC  P0
4e2: 00 00     DEC  P0
4e4: 00 00     DEC  P0
4e6: 00 00     DEC  P0
4e8: 00 00     DEC  P0
4ea: 00 00     DEC  P0
4ec: 00 00     DEC  P0
4ee: 00 00     DEC  P0
4f0: 00 00     DEC  P0
4f2: 00 00     DEC  P0
4f4: 00 00     DEC  P0
4f6: 00 00     DEC  P0
4f8: 00 00     DEC  P0
4fa: 00 00     DEC  P0
4fc: 00 00     DEC  P0
4fe: 00 00     DEC  P0
500: 00 00     DEC  P0
502: 00 00     DEC  P0
504: 00 00     DEC  P0
506: 00 00     DEC  P0
508: 00 00     DEC  P0
50a: 00 00     DEC  P0
50c: 00 00     DEC  P0
50e: 00 00     DEC  P0
510: 00 00     DEC  P0
512: 00 00     DEC  P0
514: 00 00     DEC  P0
516: 00 00     DEC  P0
518: 00 00     DEC  P0
51a: 00 00     DEC  P0
51c: 00 00     DEC  P0
51e: 00 00     DEC  P0
520: 00 00     DEC  P0
522: 00 00     DEC  P0
524: 00 00     DEC  P0
526: 00 00     DEC  P0
528: 00 00     DEC  P0
52a: 00 00     DEC  P0
52c: 00 00     DEC  P0
52e: 00 00     DEC  P0
530: 00 00     DEC  P0
532: 00 00     DEC  P0
534: 00 00     DEC  P0
536: 00 00     DEC  P0
538: 00 00     DEC  P0
53a: 00 00     DEC  P0
53c: 00 00     DEC  P0
53e: 00 00     DEC  P0
540: 00 00     DEC  P0
542: 00 00     DEC  P0
544: 00 00     DEC  P0
546: 00 00     DEC  P0
548: 00 00     DEC  P0
54a: 00 00     DEC  P0
54c: 00 00     DEC  P0
54e: 00 00     DEC  P0
550: 00 00     DEC  P0
552: 00 00     DEC  P0
554: 00 00     DEC  P0
556: 00 00     DEC  P0
558: 00 00     DEC  P0
55a: 00 00     DEC  P0
55c: 00 00     DEC  P0
55e: 00 00     DEC  P0
560: 00 00     DEC  P0
562: 00 00     DEC  P0
564: 00 00     DEC  P0
566: 00 00     DEC  P0
568: 00 00     DEC  P0
56a: 00 00     DEC  P0
56c: 00 00     DEC  P0
56e: 00 00     DEC  P0
570: 00 00     DEC  P0
572: 00 00     DEC  P0
574: 00 00     DEC  P0
576: 00 00     DEC  P0
578: 00 00     DEC  P0
57a: 00 00     DEC  P0
57c: 00 00     DEC  P0
57e: 00 00     DEC  P0
580: 00 00     DEC  P0
582: 00 00     DEC  P0
584: 00 00     DEC  P0
586: 00 00     DEC  P0
588: 00 00     DEC  P0
58a: 00 00     DEC  P0
58c: 00 00     DEC  P0
58e: 00 00     DEC  P0
590: 00 00     DEC  P0
592: 00 00     DEC  P0
594: 00 00     DEC  P0
596: 00 00     DEC  P0
598: 00 00     DEC  P0
59a: 00 00     DEC  P0
59c: 00 00     DEC  P0
59e: 00 00     DEC  P0
5a0: 00 00     DEC  P0
5a2: 00 00     DEC  P0
5a4: 00 00     DEC  P0
5a6: 00 00     DEC  P0
5a8: 00 00     DEC  P0
5aa: 00 00     DEC  P0
5ac: 00 00     DEC  P0
5ae: 00 00     DEC  P0
5b0: 00 00     DEC  P0
5b2: 00 00     DEC  P0
5b4: 00 00     DEC  P0
5b6: 00 00     DEC  P0
5b8: 00 00     DEC  P0
5ba: 00 00     DEC  P0
5bc: 00 00     DEC  P0
5be: 00 00     DEC  P0
5c0: 00 00     DEC  P0
5c2: 00 00     DEC  P0
5c4: 00 00     DEC  P0
5c6: 00 00     DEC  P0
5c8: 00 00     DEC  P0
5ca: 00 00     DEC  P0
5cc: 00 00     DEC  P0
5ce: 00 00     DEC  P0
5d0: 00 00     DEC  P0
5d2: 00 00     DEC  P0
5d4: 00 00     DEC  P0
5d6: 00 00     DEC  P0
5d8: 00 00     DEC  P0
5da: 00 00     DEC  P0
5dc: 00 00     DEC  P0
5de: 00 00     DEC  P0
5e0: 00 00     DEC  P0
5e2: 00 00     DEC  P0
5e4: 00 00     DEC  P0
5e6: 00 00     DEC  P0
5e8: 00 00     DEC  P0
5ea: 00 00     DEC  P0
5ec: 00 00     DEC  P0
5ee: 00 00     DEC  P0
5f0: 00 00     DEC  P0
5f2: 00 00     DEC  P0
5f4: 00 00     DEC  P0
5f6: 00 00     DEC  P0
5f8: 00 00     DEC  P0
5fa: 00 00     DEC  P0
5fc: 00 00     DEC  P0
5fe: 00 00     DEC  P0
600: 00 00     DEC  P0
602: 00 00     DEC  P0
604: 00 00     DEC  P0
606: 00 00     DEC  P0
608: 00 00     DEC  P0
60a: 00 00     DEC  P0
60c: 00 00     DEC  P0
60e: 00 00     DEC  P0
610: 00 00     DEC  P0
612: 00 00     DEC  P0
614: 00 00     DEC  P0
616: 00 00     DEC  P0
618: 00 00     DEC  P0
61a: 00 00     DEC  P0
61c: 00 00     DEC  P0
61e: 00 00     DEC  P0
620: 00 00     DEC  P0
622: 00 00     DEC  P0
624: 00 00     DEC  P0
626: 00 00     DEC  P0
628: 00 00     DEC  P0
62a: 00 00     DEC  P0
62c: 00 00     DEC  P0
62e: 00 00     DEC  P0
630: 00 00     DEC  P0
632: 00 00     DEC  P0
634: 00 00     DEC  P0
636: 00 00     DEC  P0
638: 00 00     DEC  P0
63a: 00 00     DEC  P0
63c: 00 00     DEC  P0
63e: 00 00     DEC  P0
640: 00 00     DEC  P0
642: 00 00     DEC  P0
644: 00 00     DEC  P0
646: 00 00     DEC  P0
648: 00 00     DEC  P0
64a: 00 00     DEC  P0
64c: 00 00     DEC  P0
64e: 00 00     DEC  P0
650: 00 00     DEC  P0
652: 00 00     DEC  P0
654: 00 00     DEC  P0
656: 00 00     DEC  P0
658: 00 00     DEC  P0
65a: 00 00     DEC  P0
65c: 00 00     DEC  P0
65e: 00 00     DEC  P0
660: 00 00     DEC  P0
662: 00 00     DEC  P0
664: 00 00     DEC  P0
666: 00 00     DEC  P0
668: 00 00     DEC  P0
66a: 00 00     DEC  P0
66c: 00 00     DEC  P0
66e: 00 00     DEC  P0
670: 00 00     DEC  P0
672: 00 00     DEC  P0
674: 00 00     DEC  P0
676: 00 00     DEC  P0
678: 00 00     DEC  P0
67a: 00 00     DEC  P0
67c: 00 00     DEC  P0
67e: 00 00     DEC  P0
680: 00 00     DEC  P0
682: 00 00     DEC  P0
684: 00 00     DEC  P0
686: 00 00     DEC  P0
688: 00 00     DEC  P0
68a: 00 00     DEC  P0
68c: 00 00     DEC  P0
68e: 00 00     DEC  P0
690: 00 00     DEC  P0
692: 00 00     DEC  P0
694: 00 00     DEC  P0
696: 00 00     DEC  P0
698: 00 00     DEC  P0
69a: 00 00     DEC  P0
69c: 00 00     DEC  P0
69e: 00 00     DEC  P0
6a0: 00 00     DEC  P0
6a2: 00 00     DEC  P0
6a4: 00 00     DEC  P0
6a6: 00 00     DEC  P0
6a8: 00 00     DEC  P0
6aa: 00 00     DEC  P0
6ac: 00 00     DEC  P0
6ae: 00 00     DEC  P0
6b0: 00 00     DEC  P0
6b2: 00 00     DEC  P0
6b4: 00 00     DEC  P0
6b6: 00 00     DEC  P0
6b8: 00 00     DEC  P0
6ba: 00 00     DEC  P0
6bc: 00 00     DEC  P0
6be: 00 00     DEC  P0
6c0: 00 00     DEC  P0
6c2: 00 00     DEC  P0
6c4: 00 00     DEC  P0
6c6: 00 00     DEC  P0
6c8: 00 00     DEC  P0
6ca: 00 00     DEC  P0
6cc: 00 00     DEC  P0
6ce: 00 00     DEC  P0
6d0: 00 00     DEC  P0
6d2: 00 00     DEC  P0
6d4: 00 00     DEC  P0
6d6: 00 00     DEC  P0
6d8: 00 00     DEC  P0
6da: 00 00     DEC  P0
6dc: 00 00     DEC  P0
6de: 00 00     DEC  P0
6e0: 00 00     DEC  P0
6e2: 00 00     DEC  P0
6e4: 00 00     DEC  P0
6e6: 00 00     DEC  P0
6e8: 00 00     DEC  P0
6ea: 00 00     DEC  P0
6ec: 00 00     DEC  P0
6ee: 00 00     DEC  P0
6f0: 00 00     DEC  P0
6f2: 00 00     DEC  P0
6f4: 00 00     DEC  P0
6f6: 00 00     DEC  P0
6f8: 00 00     DEC  P0
6fa: 00 00     DEC  P0
6fc: 00 00     DEC  P0
6fe: 00 00     DEC  P0
700: 00 00     DEC  P0
702: 00 00     DEC  P0
704: 00 00     DEC  P0
706: 00 00     DEC  P0
708: 00 00     DEC  P0
70a: 00 00     DEC  P0
70c: 00 00     DEC  P0
70e: 00 00     DEC  P0
710: 00 00     DEC  P0
712: 00 00     DEC  P0
714: 00 00     DEC  P0
716: 00 00     DEC  P0
718: 00 00     DEC  P0
71a: 00 00     DEC  P0
71c: 00 00     DEC  P0
71e: 00 00     DEC  P0
720: 00 00     DEC  P0
722: 00 00     DEC  P0
724: 00 00     DEC  P0
726: 00 00     DEC  P0
728: 00 00     DEC  P0
72a: 00 00     DEC  P0
72c: 00 00     DEC  P0
72e: 00 00     DEC  P0
730: 00 00     DEC  P0
732: 00 00     DEC  P0
734: 00 00     DEC  P0
736: 00 00     DEC  P0
738: 00 00     DEC  P0
73a: 00 00     DEC  P0
73c: 00 00     DEC  P0
73e: 00 00     DEC  P0
740: 00 00     DEC  P0
742: 00 00     DEC  P0
744: 00 00     DEC  P0
746: 00 00     DEC  P0
748: 00 00     DEC  P0
74a: 00 00     DEC  P0
74c: 00 00     DEC  P0
74e: 00 00     DEC  P0
750: 00 00     DEC  P0
752: 00 00     DEC  P0
754: 00 00     DEC  P0
756: 00 00     DEC  P0
758: 00 00     DEC  P0
75a: 00 00     DEC  P0
75c: 00 00     DEC  P0
75e: 00 00     DEC  P0
760: 00 00     DEC  P0
762: 00 00     DEC  P0
764: 00 00     DEC  P0
766: 00 00     DEC  P0
768: 00 00     DEC  P0
76a: 00 00     DEC  P0
76c: 00 00     DEC  P0
76e: 00 00     DEC  P0
770: 00 00     DEC  P0
772: 00 00     DEC  P0
774: 00 00     DEC  P0
776: 00 00     DEC  P0
778: 00 00     DEC  P0
77a: 00 00     DEC  P0
77c: 00 00     DEC  P0
77e: 00 00     DEC  P0
780: 00 00     DEC  P0
782: 00 00     DEC  P0
784: 00 00     DEC  P0
786: 00 00     DEC  P0
788: 00 00     DEC  P0
78a: 00 00     DEC  P0
78c: 00 00     DEC  P0
78e: 00 00     DEC  P0
790: 00 00     DEC  P0
792: 00 00     DEC  P0
794: 00 00     DEC  P0
796: 00 00     DEC  P0
798: 00 00     DEC  P0
79a: 00 00     DEC  P0
79c: 00 00     DEC  P0
79e: 00 00     DEC  P0
7a0: 00 00     DEC  P0
7a2: 00 00     DEC  P0
7a4: 00 00     DEC  P0
7a6: 00 00     DEC  P0
7a8: 00 00     DEC  P0
7aa: 00 00     DEC  P0
7ac: 00 00     DEC  P0
7ae: 00 00     DEC  P0
7b0: 00 00     DEC  P0
7b2: 00 00     DEC  P0
7b4: 00 00     DEC  P0
7b6: 00 00     DEC  P0
7b8: 00 00     DEC  P0
7ba: 00 00     DEC  P0
7bc: 00 00     DEC  P0
7be: 00 00     DEC  P0
7c0: 00 00     DEC  P0
7c2: 00 00     DEC  P0
7c4: 00 00     DEC  P0
7c6: 00 00     DEC  P0
7c8: 00 00     DEC  P0
7ca: 00 00     DEC  P0
7cc: 00 00     DEC  P0
7ce: 00 00     DEC  P0
7d0: 00 00     DEC  P0
7d2: 00 00     DEC  P0
7d4: 00 00     DEC  P0
7d6: 00 00     DEC  P0
7d8: 00 00     DEC  P0
7da: 00 00     DEC  P0
7dc: 00 00     DEC  P0
7de: 00 00     DEC  P0
7e0: 00 00     DEC  P0
7e2: 00 00     DEC  P0
7e4: 00 00     DEC  P0
7e6: 00 00     DEC  P0
7e8: 00 00     DEC  P0
7ea: 00 00     DEC  P0
7ec: 00 00     DEC  P0
7ee: 00 00     DEC  P0
7f0: 00 00     DEC  P0
7f2: 00 00     DEC  P0
7f4: 00 00     DEC  P0
7f6: 00 00     DEC  P0
7f8: 00 00     DEC  P0
7fa: 00 00     DEC  P0
7fc: 00 00     DEC  P0
7fe: 00 00     DEC  P0
800: 00 00     DEC  P0
802: 00 00     DEC  P0
804: 00 00     DEC  P0
806: 00 00     DEC  P0
808: 00 00     DEC  P0
80a: 00 00     DEC  P0
80c: 00 00     DEC  P0
80e: 00 00     DEC  P0
810: 00 00     DEC  P0
812: 00 00     DEC  P0
814: 00 00     DEC  P0
816: 00 00     DEC  P0
818: 00 00     DEC  P0
81a: 00 00     DEC  P0
81c: 00 00     DEC  P0
81e: 00 00     DEC  P0
820: 00 00     DEC  P0
822: 00 00     DEC  P0
824: 00 00     DEC  P0
826: 00 00     DEC  P0
828: 00 00     DEC  P0
82a: 00 00     DEC  P0
82c: 00 00     DEC  P0
82e: 00 00     DEC  P0
830: 00 00     DEC  P0
832: 00 00     DEC  P0
834: 00 00     DEC  P0
836: 00 00     DEC  P0
838: 00 00     DEC  P0
83a: 00 00     DEC  P0
83c: 00 00     DEC  P0
83e: 00 00     DEC  P0
840: 00 00     DEC  P0
842: 00 00     DEC  P0
844: 00 00     DEC  P0
846: 00 00     DEC  P0
848: 00 00     DEC  P0
84a: 00 00     DEC  P0
84c: 00 00     DEC  P0
84e: 00 00     DEC  P0
850: 00 00     DEC  P0
852: 00 00     DEC  P0
854: 00 00     DEC  P0
856: 00 00     DEC  P0
858: 00 00     DEC  P0
85a: 00 00     DEC  P0
85c: 00 00     DEC  P0
85e: 00 00     DEC  P0
860: 00 00     DEC  P0
862: 00 00     DEC  P0
864: 00 00     DEC  P0
866: 00 00     DEC  P0
868: 00 00     DEC  P0
86a: 00 00     DEC  P0
86c: 00 00     DEC  P0
86e: 00 00     DEC  P0
870: 00 00     DEC  P0
872: 00 00     DEC  P0
874: 00 00     DEC  P0
876: 00 00     DEC  P0
878: 00 00     DEC  P0
87a: 00 00     DEC  P0
87c: 00 00     DEC  P0
87e: 00 00     DEC  P0
880: 00 00     DEC  P0
882: 00 00     DEC  P0
884: 00 00     DEC  P0
886: 00 00     DEC  P0
888: 00 00     DEC  P0
88a: 00 00     DEC  P0
88c: 00 00     DEC  P0
88e: 00 00     DEC  P0
890: 00 00     DEC  P0
892: 00 00     DEC  P0
894: 00 00     DEC  P0
896: 00 00     DEC  P0
898: 00 00     DEC  P0
89a: 00 00     DEC  P0
89c: 00 00     DEC  P0
89e: 00 00     DEC  P0
8a0: 00 00     DEC  P0
8a2: 00 00     DEC  P0
8a4: 00 00     DEC  P0
8a6: 00 00     DEC  P0
8a8: 00 00     DEC  P0
8aa: 00 00     DEC  P0
8ac: 00 00     DEC  P0
8ae: 00 00     DEC  P0
8b0: 00 00     DEC  P0
8b2: 00 00     DEC  P0
8b4: 00 00     DEC  P0
8b6: 00 00     DEC  P0
8b8: 00 00     DEC  P0
8ba: 00 00     DEC  P0
8bc: 00 00     DEC  P0
8be: 00 00     DEC  P0
8c0: 00 00     DEC  P0
8c2: 00 00     DEC  P0
8c4: 00 00     DEC  P0
8c6: 00 00     DEC  P0
8c8: 00 00     DEC  P0
8ca: 00 00     DEC  P0
8cc: 00 00     DEC  P0
8ce: 00 00     DEC  P0
8d0: 00 00     DEC  P0
8d2: 00 00     DEC  P0
8d4: 00 00     DEC  P0
8d6: 00 00     DEC  P0
8d8: 00 00     DEC  P0
8da: 00 00     DEC  P0
8dc: 00 00     DEC  P0
8de: 00 00     DEC  P0
8e0: 00 00     DEC  P0
8e2: 00 00     DEC  P0
8e4: 00 00     DEC  P0
8e6: 00 00     DEC  P0
8e8: 00 00     DEC  P0
8ea: 00 00     DEC  P0
8ec: 00 00     DEC  P0
8ee: 00 00     DEC  P0
8f0: 00 00     DEC  P0
8f2: 00 00     DEC  P0
8f4: 00 00     DEC  P0
8f6: 00 00     DEC  P0
8f8: 00 00     DEC  P0
8fa: 00 00     DEC  P0
8fc: 00 00     DEC  P0
8fe: 00 00     DEC  P0
900: 00 00     DEC  P0
902: 00 00     DEC  P0
904: 00 00     DEC  P0
906: 00 00     DEC  P0
908: 00 00     DEC  P0
90a: 00 00     DEC  P0
90c: 00 00     DEC  P0
90e: 00 00     DEC  P0
910: 00 00     DEC  P0
912: 00 00     DEC  P0
914: 00 00     DEC  P0
916: 00 00     DEC  P0
918: 00 00     DEC  P0
91a: 00 00     DEC  P0
91c: 00 00     DEC  P0
91e: 00 00     DEC  P0
920: 00 00     DEC  P0
922: 00 00     DEC  P0
924: 00 00     DEC  P0
926: 00 00     DEC  P0
928: 00 00     DEC  P0
92a: 00 00     DEC  P0
92c: 00 00     DEC  P0
92e: 00 00     DEC  P0
930: 00 00     DEC  P0
932: 00 00     DEC  P0
934: 00 00     DEC  P0
936: 00 00     DEC  P0
938: 00 00     DEC  P0
93a: 00 00     DEC  P0
93c: 00 00     DEC  P0
93e: 00 00     DEC  P0
940: 00 00     DEC  P0
942: 00 00     DEC  P0
944: 00 00     DEC  P0
946: 00 00     DEC  P0
948: 00 00     DEC  P0
94a: 00 00     DEC  P0
94c: 00 00     DEC  P0
94e: 00 00     DEC  P0
950: 00 00     DEC  P0
952: 00 00     DEC  P0
954: 00 00     DEC  P0
956: 00 00     DEC  P0
958: 00 00     DEC  P0
95a: 00 00     DEC  P0
95c: 00 00     DEC  P0
95e: 00 00     DEC  P0
960: 00 00     DEC  P0
962: 00 00     DEC  P0
964: 00 00     DEC  P0
966: 00 00     DEC  P0
968: 00 00     DEC  P0
96a: 00 00     DEC  P0
96c: 00 00     DEC  P0
96e: 00 00     DEC  P0
970: 00 00     DEC  P0
972: 00 00     DEC  P0
974: 00 00     DEC  P0
976: 00 00     DEC  P0
978: 00 00     DEC  P0
97a: 00 00     DEC  P0
97c: 00 00     DEC  P0
97e: 00 00     DEC  P0
980: 00 00     DEC  P0
982: 00 00     DEC  P0
984: 00 00     DEC  P0
986: 00 00     DEC  P0
988: 00 00     DEC  P0
98a: 00 00     DEC  P0
98c: 00 00     DEC  P0
98e: 00 00     DEC  P0
990: 00 00     DEC  P0
992: 00 00     DEC  P0
994: 00 00     DEC  P0
996: 00 00     DEC  P0
998: 00 00     DEC  P0
99a: 00 00     DEC  P0
99c: 00 00     DEC  P0
99e: 00 00     DEC  P0
9a0: 00 00     DEC  P0
9a2: 00 00     DEC  P0
9a4: 00 00     DEC  P0
9a6: 00 00     DEC  P0
9a8: 00 00     DEC  P0
9aa: 00 00     DEC  P0
9ac: 00 00     DEC  P0
9ae: 00 00     DEC  P0
9b0: 00 00     DEC  P0
9b2: 00 00     DEC  P0
9b4: 00 00     DEC  P0
9b6: 00 00     DEC  P0
9b8: 00 00     DEC  P0
9ba: 00 00     DEC  P0
9bc: 00 00     DEC  P0
9be: 00 00     DEC  P0
9c0: 00 00     DEC  P0
9c2: 00 00     DEC  P0
9c4: 00 00     DEC  P0
9c6: 00 00     DEC  P0
9c8: 00 00     DEC  P0
9ca: 00 00     DEC  P0
9cc: 00 00     DEC  P0
9ce: 00 00     DEC  P0
9d0: 00 00     DEC  P0
9d2: 00 00     DEC  P0
9d4: 00 00     DEC  P0
9d6: 00 00     DEC  P0
9d8: 00 00     DEC  P0
9da: 00 00     DEC  P0
9dc: 00 00     DEC  P0
9de: 00 00     DEC  P0
9e0: 00 00     DEC  P0
9e2: 00 00     DEC  P0
9e4: 00 00     DEC  P0
9e6: 00 00     DEC  P0
9e8: 00 00     DEC  P0
9ea: 00 00     DEC  P0
9ec: 00 00     DEC  P0
9ee: 00 00     DEC  P0
9f0: 00 00     DEC  P0
9f2: 00 00     DEC  P0
9f4: 00 00     DEC  P0
9f6: 00 00     DEC  P0
9f8: 00 00     DEC  P0
9fa: 00 00     DEC  P0
9fc: 00 00     DEC  P0
9fe: 00 00     DEC  P0
a00: 00 00     DEC  P0
a02: 00 00     DEC  P0
a04: 00 00     DEC  P0
a06: 00 00     DEC  P0
a08: 00 00     DEC  P0
a0a: 00 00     DEC  P0
a0c: 00 00     DEC  P0
a0e: 00 00     DEC  P0
a10: 00 00     DEC  P0
a12: 00 00     DEC  P0
a14: 00 00     DEC  P0
a16: 00 00     DEC  P0
a18: 00 00     DEC  P0
a1a: 00 00     DEC  P0
a1c: 00 00     DEC  P0
a1e: 00 00     DEC  P0
a20: 00 00     DEC  P0
a22: 00 00     DEC  P0
a24: 00 00     DEC  P0
a26: 00 00     DEC  P0
a28: 00 00     DEC  P0
a2a: 00 00     DEC  P0
a2c: 00 00     DEC  P0
a2e: 00 00     DEC  P0
a30: 00 00     DEC  P0
a32: 00 00     DEC  P0
a34: 00 00     DEC  P0
a36: 00 00     DEC  P0
a38: 00 00     DEC  P0
a3a: 00 00     DEC  P0
a3c: 00 00     DEC  P0
a3e: 00 00     DEC  P0
a40: 00 00     DEC  P0
a42: 00 00     DEC  P0
a44: 00 00     DEC  P0
a46: 00 00     DEC  P0
a48: 00 00     DEC  P0
a4a: 00 00     DEC  P0
a4c: 00 00     DEC  P0
a4e: 00 00     DEC  P0
a50: 00 00     DEC  P0
a52: 00 00     DEC  P0
a54: 00 00     DEC  P0
a56: 00 00     DEC  P0
a58: 00 00     DEC  P0
a5a: 00 00     DEC  P0
a5c: 00 00     DEC  P0
a5e: 00 00     DEC  P0
a60: 00 00     DEC  P0
a62: 00 00     DEC  P0
a64: 00 00     DEC  P0
a66: 00 00     DEC  P0
a68: 00 00     DEC  P0
a6a: 00 00     DEC  P0
a6c: 00 00     DEC  P0
a6e: 00 00     DEC  P0
a70: 00 00     DEC  P0
a72: 00 00     DEC  P0
a74: 00 00     DEC  P0
a76: 00 00     DEC  P0
a78: 00 00     DEC  P0
a7a: 00 00     DEC  P0
a7c: 00 00     DEC  P0
a7e: 00 00     DEC  P0
a80: 00 00     DEC  P0
a82: 00 00     DEC  P0
a84: 00 00     DEC  P0
a86: 00 00     DEC  P0
a88: 00 00     DEC  P0
a8a: 00 00     DEC  P0
a8c: 00 00     DEC  P0
a8e: 00 00     DEC  P0
a90: 00 00     DEC  P0
a92: 00 00     DEC  P0
a94: 00 00     DEC  P0
a96: 00 00     DEC  P0
a98: 00 00     DEC  P0
a9a: 00 00     DEC  P0
a9c: 00 00     DEC  P0
a9e: 00 00     DEC  P0
aa0: 00 00     DEC  P0
aa2: 00 00     DEC  P0
aa4: 00 00     DEC  P0
aa6: 00 00     DEC  P0
aa8: 00 00     DEC  P0
aaa: 00 00     DEC  P0
aac: 00 00     DEC  P0
aae: 00 00     DEC  P0
ab0: 00 00     DEC  P0
ab2: 00 00     DEC  P0
ab4: 00 00     DEC  P0
ab6: 00 00     DEC  P0
ab8: 00 00     DEC  P0
aba: 00 00     DEC  P0
abc: 00 00     DEC  P0
abe: 00 00     DEC  P0
ac0: 00 00     DEC  P0
ac2: 00 00     DEC  P0
ac4: 00 00     DEC  P0
ac6: 00 00     DEC  P0
ac8: 00 00     DEC  P0
aca: 00 00     DEC  P0
acc: 00 00     DEC  P0
ace: 00 00     DEC  P0
ad0: 00 00     DEC  P0
ad2: 00 00     DEC  P0
ad4: 00 00     DEC  P0
ad6: 00 00     DEC  P0
ad8: 00 00     DEC  P0
ada: 00 00     DEC  P0
adc: 00 00     DEC  P0
ade: 00 00     DEC  P0
ae0: 00 00     DEC  P0
ae2: 00 00     DEC  P0
ae4: 00 00     DEC  P0
ae6: 00 00     DEC  P0
ae8: 00 00     DEC  P0
aea: 00 00     DEC  P0
aec: 00 00     DEC  P0
aee: 00 00     DEC  P0
af0: 00 00     DEC  P0
af2: 00 00     DEC  P0
af4: 00 00     DEC  P0
af6: 00 00     DEC  P0
af8: 00 00     DEC  P0
afa: 00 00     DEC  P0
afc: 00 00     DEC  P0
afe: 00 00     DEC  P0
b00: 00 00     DEC  P0
b02: 00 00     DEC  P0
b04: 00 00     DEC  P0
b06: 00 00     DEC  P0
b08: 00 00     DEC  P0
b0a: 00 00     DEC  P0
b0c: 00 00     DEC  P0
b0e: 00 00     DEC  P0
b10: 00 00     DEC  P0
b12: 00 00     DEC  P0
b14: 00 00     DEC  P0
b16: 00 00     DEC  P0
b18: 00 00     DEC  P0
b1a: 00 00     DEC  P0
b1c: 00 00     DEC  P0
b1e: 00 00     DEC  P0
b20: 00 00     DEC  P0
b22: 00 00     DEC  P0
b24: 00 00     DEC  P0
b26: 00 00     DEC  P0
b28: 00 00     DEC  P0
b2a: 00 00     DEC  P0
b2c: 00 00     DEC  P0
b2e: 00 00     DEC  P0
b30: 00 00     DEC  P0
b32: 00 00     DEC  P0
b34: 00 00     DEC  P0
b36: 00 00     DEC  P0
b38: 00 00     DEC  P0
b3a: 00 00     DEC  P0
b3c: 00 00     DEC  P0
b3e: 00 00     DEC  P0
b40: 00 00     DEC  P0
b42: 00 00     DEC  P0
b44: 00 00     DEC  P0
b46: 00 00     DEC  P0
b48: 00 00     DEC  P0
b4a: 00 00     DEC  P0
b4c: 00 00     DEC  P0
b4e: 00 00     DEC  P0
b50: 00 00     DEC  P0
b52: 00 00     DEC  P0
b54: 00 00     DEC  P0
b56: 00 00     DEC  P0
b58: 00 00     DEC  P0
b5a: 00 00     DEC  P0
b5c: 00 00     DEC  P0
b5e: 00 00     DEC  P0
b60: 00 00     DEC  P0
b62: 00 00     DEC  P0
b64: 00 00     DEC  P0
b66: 00 00     DEC  P0
b68: 00 00     DEC  P0
b6a: 00 00     DEC  P0
b6c: 00 00     DEC  P0
b6e: 00 00     DEC  P0
b70: 00 00     DEC  P0
b72: 00 00     DEC  P0
b74: 00 00     DEC  P0
b76: 00 00     DEC  P0
b78: 00 00     DEC  P0
b7a: 00 00     DEC  P0
b7c: 00 00     DEC  P0
b7e: 00 00     DEC  P0
b80: 00 00     DEC  P0
b82: 00 00     DEC  P0
b84: 00 00     DEC  P0
b86: 00 00     DEC  P0
b88: 00 00     DEC  P0
b8a: 00 00     DEC  P0
b8c: 00 00     DEC  P0
b8e: 00 00     DEC  P0
b90: 00 00     DEC  P0
b92: 00 00     DEC  P0
b94: 00 00     DEC  P0
b96: 00 00     DEC  P0
b98: 00 00     DEC  P0
b9a: 00 00     DEC  P0
b9c: 00 00     DEC  P0
b9e: 00 00     DEC  P0
ba0: 00 00     DEC  P0
ba2: 00 00     DEC  P0
ba4: 00 00     DEC  P0
ba6: 00 00     DEC  P0
ba8: 00 00     DEC  P0
baa: 00 00     DEC  P0
bac: 00 00     DEC  P0
bae: 00 00     DEC  P0
bb0: 00 00     DEC  P0
bb2: 00 00     DEC  P0
bb4: 00 00     DEC  P0
bb6: 00 00     DEC  P0
bb8: 00 00     DEC  P0
bba: 00 00     DEC  P0
bbc: 00 00     DEC  P0
bbe: 00 00     DEC  P0
bc0: 00 00     DEC  P0
bc2: 00 00     DEC  P0
bc4: 00 00     DEC  P0
bc6: 00 00     DEC  P0
bc8: 00 00     DEC  P0
bca: 00 00     DEC  P0
bcc: 00 00     DEC  P0
bce: 00 00     DEC  P0
bd0: 00 00     DEC  P0
bd2: 00 00     DEC  P0
bd4: 00 00     DEC  P0
bd6: 00 00     DEC  P0
bd8: 00 00     DEC  P0
bda: 00 00     DEC  P0
bdc: 00 00     DEC  P0
bde: 00 00     DEC  P0
be0: 00 00     DEC  P0
be2: 00 00     DEC  P0
be4: 00 00     DEC  P0
be6: 00 00     DEC  P0
be8: 00 00     DEC  P0
bea: 00 00     DEC  P0
bec: 00 00     DEC  P0
bee: 00 00     DEC  P0
bf0: 00 00     DEC  P0
bf2: 00 00     DEC  P0
bf4: 00 00     DEC  P0
bf6: 00 00     DEC  P0
bf8: 00 00     DEC  P0
bfa: 00 00     DEC  P0
bfc: 00 00     DEC  P0
bfe: 00 00     DEC  P0
c00: 00 00     DEC  P0
c02: 00 00     DEC  P0
c04: 00 00     DEC  P0
c06: 00 00     DEC  P0
c08: 00 00     DEC  P0
c0a: 00 00     DEC  P0
c0c: 00 00     DEC  P0
c0e: 00 00     DEC  P0
c10: 00 00     DEC  P0
c12: 00 00     DEC  P0
c14: 00 00     DEC  P0
c16: 00 00     DEC  P0
c18: 00 00     DEC  P0
c1a: 00 00     DEC  P0
c1c: 00 00     DEC  P0
c1e: 00 00     DEC  P0
c20: 00 00     DEC  P0
c22: 00 00     DEC  P0
c24: 00 00     DEC  P0
c26: 00 00     DEC  P0
c28: 00 00     DEC  P0
c2a: 00 00     DEC  P0
c2c: 00 00     DEC  P0
c2e: 00 00     DEC  P0
c30: 00 00     DEC  P0
c32: 00 00     DEC  P0
c34: 00 00     DEC  P0
c36: 00 00     DEC  P0
c38: 00 00     DEC  P0
c3a: 00 00     DEC  P0
c3c: 00 00     DEC  P0
c3e: 00 00     DEC  P0
c40: 00 00     DEC  P0
c42: 00 00     DEC  P0
c44: 00 00     DEC  P0
c46: 00 00     DEC  P0
c48: 00 00     DEC  P0
c4a: 00 00     DEC  P0
c4c: 00 00     DEC  P0
c4e: 00 00     DEC  P0
c50: 00 00     DEC  P0
c52: 00 00     DEC  P0
c54: 00 00     DEC  P0
c56: 00 00     DEC  P0
c58: 00 00     DEC  P0
c5a: 00 00     DEC  P0
c5c: 00 00     DEC  P0
c5e: 00 00     DEC  P0
c60: 00 00     DEC  P0
c62: 00 00     DEC  P0
c64: 00 00     DEC  P0
c66: 00 00     DEC  P0
c68: 00 00     DEC  P0
c6a: 00 00     DEC  P0
c6c: 00 00     DEC  P0
c6e: 00 00     DEC  P0
c70: 00 00     DEC  P0
c72: 00 00     DEC  P0
c74: 00 00     DEC  P0
c76: 00 00     DEC  P0
c78: 00 00     DEC  P0
c7a: 00 00     DEC  P0
c7c: 00 00     DEC  P0
c7e: 00 00     DEC  P0
c80: 00 00     DEC  P0
c82: 00 00     DEC  P0
c84: 00 00     DEC  P0
c86: 00 00     DEC  P0
c88: 00 00     DEC  P0
c8a: 00 00     DEC  P0
c8c: 00 00     DEC  P0
c8e: 00 00     DEC  P0
c90: 00 00     DEC  P0
c92: 00 00     DEC  P0
c94: 00 00     DEC  P0
c96: 00 00     DEC  P0
c98: 00 00     DEC  P0
c9a: 00 00     DEC  P0
c9c: 00 00     DEC  P0
c9e: 00 00     DEC  P0
ca0: 00 00     DEC  P0
ca2: 00 00     DEC  P0
ca4: 00 00     DEC  P0
ca6: 00 00     DEC  P0
ca8: 00 00     DEC  P0
caa: 00 00     DEC  P0
cac: 00 00     DEC  P0
cae: 00 00     DEC  P0
cb0: 00 00     DEC  P0
cb2: 00 00     DEC  P0
cb4: 00 00     DEC  P0
cb6: 00 00     DEC  P0
cb8: 00 00     DEC  P0
cba: 00 00     DEC  P0
cbc: 00 00     DEC  P0
cbe: 00 00     DEC  P0
cc0: 00 00     DEC  P0
cc2: 00 00     DEC  P0
cc4: 00 00     DEC  P0
cc6: 00 00     DEC  P0
cc8: 00 00     DEC  P0
cca: 00 00     DEC  P0
ccc: 00 00     DEC  P0
cce: 00 00     DEC  P0
cd0: 00 00     DEC  P0
cd2: 00 00     DEC  P0
cd4: 00 00     DEC  P0
cd6: 00 00     DEC  P0
cd8: 00 00     DEC  P0
cda: 00 00     DEC  P0
cdc: 00 00     DEC  P0
cde: 00 00     DEC  P0
ce0: 00 00     DEC  P0
ce2: 00 00     DEC  P0
ce4: 00 00     DEC  P0
ce6: 00 00     DEC  P0
ce8: 00 00     DEC  P0
cea: 00 00     DEC  P0
cec: 00 00     DEC  P0
cee: 00 00     DEC  P0
cf0: 00 00     DEC  P0
cf2: 00 00     DEC  P0
cf4: 00 00     DEC  P0
cf6: 00 00     DEC  P0
cf8: 00 00     DEC  P0
cfa: 00 00     DEC  P0
cfc: 00 00     DEC  P0
cfe: 00 00     DEC  P0
d00: 00 00     DEC  P0
d02: 00 00     DEC  P0
d04: 00 00     DEC  P0
d06: 00 00     DEC  P0
d08: 00 00     DEC  P0
d0a: 00 00     DEC  P0
d0c: 00 00     DEC  P0
d0e: 00 00     DEC  P0
d10: 00 00     DEC  P0
d12: 00 00     DEC  P0
d14: 00 00     DEC  P0
d16: 00 00     DEC  P0
d18: 00 00     DEC  P0
d1a: 00 00     DEC  P0
d1c: 00 00     DEC  P0
d1e: 00 00     DEC  P0
d20: 00 00     DEC  P0
d22: 00 00     DEC  P0
d24: 00 00     DEC  P0
d26: 00 00     DEC  P0
d28: 00 00     DEC  P0
d2a: 00 00     DEC  P0
d2c: 00 00     DEC  P0
d2e: 00 00     DEC  P0
d30: 00 00     DEC  P0
d32: 00 00     DEC  P0
d34: 00 00     DEC  P0
d36: 00 00     DEC  P0
d38: 00 00     DEC  P0
d3a: 00 00     DEC  P0
d3c: 00 00     DEC  P0
d3e: 00 00     DEC  P0
d40: 00 00     DEC  P0
d42: 00 00     DEC  P0
d44: 00 00     DEC  P0
d46: 00 00     DEC  P0
d48: 00 00     DEC  P0
d4a: 00 00     DEC  P0
d4c: 00 00     DEC  P0
d4e: 00 00     DEC  P0
d50: 00 00     DEC  P0
d52: 00 00     DEC  P0
d54: 00 00     DEC  P0
d56: 00 00     DEC  P0
d58: 00 00     DEC  P0
d5a: 00 00     DEC  P0
d5c: 00 00     DEC  P0
d5e: 00 00     DEC  P0
d60: 00 00     DEC  P0
d62: 00 00     DEC  P0
d64: 00 00     DEC  P0
d66: 00 00     DEC  P0
d68: 00 00     DEC  P0
d6a: 00 00     DEC  P0
d6c: 00 00     DEC  P0
d6e: 00 00     DEC  P0
d70: 00 00     DEC  P0
d72: 00 00     DEC  P0
d74: 00 00     DEC  P0
d76: 00 00     DEC  P0
d78: 00 00     DEC  P0
d7a: 00 00     DEC  P0
d7c: 00 00     DEC  P0
d7e: 00 00     DEC  P0
d80: 00 00     DEC  P0
d82: 00 00     DEC  P0
d84: 00 00     DEC  P0
d86: 00 00     DEC  P0
d88: 00 00     DEC  P0
d8a: 00 00     DEC  P0
d8c: 00 00     DEC  P0
d8e: 00 00     DEC  P0
d90: 00 00     DEC  P0
d92: 00 00     DEC  P0
d94: 00 00     DEC  P0
d96: 00 00     DEC  P0
d98: 00 00     DEC  P0
d9a: 00 00     DEC  P0
d9c: 00 00     DEC  P0
d9e: 00 00     DEC  P0
da0: 00 00     DEC  P0
da2: 00 00     DEC  P0
da4: 00 00     DEC  P0
da6: 00 00     DEC  P0
da8: 00 00     DEC  P0
daa: 00 00     DEC  P0
dac: 00 00     DEC  P0
dae: 00 00     DEC  P0
db0: 00 00     DEC  P0
db2: 00 00     DEC  P0
db4: 00 00     DEC  P0
db6: 00 00     DEC  P0
db8: 00 00     DEC  P0
dba: 00 00     DEC  P0
dbc: 00 00     DEC  P0
dbe: 00 00     DEC  P0
dc0: 00 00     DEC  P0
dc2: 00 00     DEC  P0
dc4: 00 00     DEC  P0
dc6: 00 00     DEC  P0
dc8: 00 00     DEC  P0
dca: 00 00     DEC  P0
dcc: 00 00     DEC  P0
dce: 00 00     DEC  P0
dd0: 00 00     DEC  P0
dd2: 00 00     DEC  P0
dd4: 00 00     DEC  P0
dd6: 00 00     DEC  P0
dd8: 00 00     DEC  P0
dda: 00 00     DEC  P0
ddc: 00 00     DEC  P0
dde: 00 00     DEC  P0
de0: 00 00     DEC  P0
de2: 00 00     DEC  P0
de4: 00 00     DEC  P0
de6: 00 00     DEC  P0
de8: 00 00     DEC  P0
dea: 00 00     DEC  P0
dec: 00 00     DEC  P0
dee: 00 00     DEC  P0
df0: 00 00     DEC  P0
df2: 00 00     DEC  P0
df4: 00 00     DEC  P0
df6: 00 00     DEC  P0
df8: 00 00     DEC  P0
dfa: 00 00     DEC  P0
dfc: 00 00     DEC  P0
dfe: 00 00     DEC  P0
e00: 00 00     DEC  P0
e02: 00 00     DEC  P0
e04: 00 00     DEC  P0
e06: 00 00     DEC  P0
e08: 00 00     DEC  P0
e0a: 00 00     DEC  P0
e0c: 00 00     DEC  P0
e0e: 00 00     DEC  P0
e10: 00 00     DEC  P0
e12: 00 00     DEC  P0
e14: 00 00     DEC  P0
e16: 00 00     DEC  P0
e18: 00 00     DEC  P0
e1a: 00 00     DEC  P0
e1c: 00 00     DEC  P0
e1e: 00 00     DEC  P0
e20: 00 00     DEC  P0
e22: 00 00     DEC  P0
e24: 00 00     DEC  P0
e26: 00 00     DEC  P0
e28: 00 00     DEC  P0
e2a: 00 00     DEC  P0
e2c: 00 00     DEC  P0
e2e: 00 00     DEC  P0
e30: 00 00     DEC  P0
e32: 00 00     DEC  P0
e34: 00 00     DEC  P0
e36: 00 00     DEC  P0
e38: 00 00     DEC  P0
e3a: 00 00     DEC  P0
e3c: 00 00     DEC  P0
e3e: 00 00     DEC  P0
e40: 00 00     DEC  P0
e42: 00 00     DEC  P0
e44: 00 00     DEC  P0
e46: 00 00     DEC  P0
e48: 00 00     DEC  P0
e4a: 00 00     DEC  P0
e4c: 00 00     DEC  P0
e4e: 00 00     DEC  P0
e50: 00 00     DEC  P0
e52: 00 00     DEC  P0
e54: 00 00     DEC  P0
e56: 00 00     DEC  P0
e58: 00 00     DEC  P0
e5a: 00 00     DEC  P0
e5c: 00 00     DEC  P0
e5e: 00 00     DEC  P0
e60: 00 00     DEC  P0
e62: 00 00     DEC  P0
e64: 00 00     DEC  P0
e66: 00 00     DEC  P0
e68: 00 00     DEC  P0
e6a: 00 00     DEC  P0
e6c: 00 00     DEC  P0
e6e: 00 00     DEC  P0
e70: 00 00     DEC  P0
e72: 00 00     DEC  P0
e74: 00 00     DEC  P0
e76: 00 00     DEC  P0
e78: 00 00     DEC  P0
e7a: 00 00     DEC  P0
e7c: 00 00     DEC  P0
e7e: 00 00     DEC  P0
e80: 00 00     DEC  P0
e82: 00 00     DEC  P0
e84: 00 00     DEC  P0
e86: 00 00     DEC  P0
e88: 00 00     DEC  P0
e8a: 00 00     DEC  P0
e8c: 00 00     DEC  P0
e8e: 00 00     DEC  P0
e90: 00 00     DEC  P0
e92: 00 00     DEC  P0
e94: 00 00     DEC  P0
e96: 00 00     DEC  P0
e98: 00 00     DEC  P0
e9a: 00 00     DEC  P0
e9c: 00 00     DEC  P0
e9e: 00 00     DEC  P0
ea0: 00 00     DEC  P0
ea2: 00 00     DEC  P0
ea4: 00 00     DEC  P0
ea6: 00 00     DEC  P0
ea8: 00 00     DEC  P0
eaa: 00 00     DEC  P0
eac: 00 00     DEC  P0
eae: 00 00     DEC  P0
eb0: 00 00     DEC  P0
eb2: 00 00     DEC  P0
eb4: 00 00     DEC  P0
eb6: 00 00     DEC  P0
eb8: 00 00     DEC  P0
eba: 00 00     DEC  P0
ebc: 00 00     DEC  P0
ebe: 00 00     DEC  P0
ec0: 00 00     DEC  P0
ec2: 00 00     DEC  P0
ec4: 00 00     DEC  P0
ec6: 00 00     DEC  P0
ec8: 00 00     DEC  P0
eca: 00 00     DEC  P0
ecc: 00 00     DEC  P0
ece: 00 00     DEC  P0
ed0: 00 00     DEC  P0
ed2: 00 00     DEC  P0
ed4: 00 00     DEC  P0
ed6: 00 00     DEC  P0
ed8: 00 00     DEC  P0
eda: 00 00     DEC  P0
edc: 00 00     DEC  P0
ede: 00 00     DEC  P0
ee0: 00 00     DEC  P0
ee2: 00 00     DEC  P0
ee4: 00 00     DEC  P0
ee6: 00 00     DEC  P0
ee8: 00 00     DEC  P0
eea: 00 00     DEC  P0
eec: 00 00     DEC  P0
eee: 00 00     DEC  P0
ef0: 00 00     DEC  P0
ef2: 00 00     DEC  P0
ef4: 00 00     DEC  P0
ef6: 00 00     DEC  P0
ef8: 00 00     DEC  P0
efa: 00 00     DEC  P0
efc: 00 00     DEC  P0
efe: 00 00     DEC  P0
f00: 00 00     DEC  P0
f02: 00 00     DEC  P0
f04: 00 00     DEC  P0
f06: 00 00     DEC  P0
f08: 00 00     DEC  P0
f0a: 00 00     DEC  P0
f0c: 00 00     DEC  P0
f0e: 00 00     DEC  P0
f10: 00 00     DEC  P0
f12: 00 00     DEC  P0
f14: 00 00     DEC  P0
f16: 00 00     DEC  P0
f18: 00 00     DEC  P0
f1a: 00 00     DEC  P0
f1c: 00 00     DEC  P0
f1e: 00 00     DEC  P0
f20: 00 00     DEC  P0
f22: 00 00     DEC  P0
f24: 00 00     DEC  P0
f26: 00 00     DEC  P0
f28: 00 00     DEC  P0
f2a: 00 00     DEC  P0
f2c: 00 00     DEC  P0
f2e: 00 00     DEC  P0
f30: 00 00     DEC  P0
f32: 00 00     DEC  P0
f34: 00 00     DEC  P0
f36: 00 00     DEC  P0
f38: 00 00     DEC  P0
f3a: 00 00     DEC  P0
f3c: 00 00     DEC  P0
f3e: 00 00     DEC  P0
f40: 00 00     DEC  P0
f42: 00 00     DEC  P0
f44: 00 00     DEC  P0
f46: 00 00     DEC  P0
f48: 00 00     DEC  P0
f4a: 00 00     DEC  P0
f4c: 00 00     DEC  P0
f4e: 00 00     DEC  P0
f50: 00 00     DEC  P0
f52: 00 00     DEC  P0
f54: 00 00     DEC  P0
f56: 00 00     DEC  P0
f58: 00 00     DEC  P0
f5a: 00 00     DEC  P0
f5c: 00 00     DEC  P0
f5e: 00 00     DEC  P0
f60: 00 00     DEC  P0
f62: 00 00     DEC  P0
f64: 00 00     DEC  P0
f66: 00 00     DEC  P0
f68: 00 00     DEC  P0
f6a: 00 00     DEC  P0
f6c: 00 00     DEC  P0
f6e: 00 00     DEC  P0
f70: 00 00     DEC  P0
f72: 00 00     DEC  P0
f74: 00 00     DEC  P0
f76: 00 00     DEC  P0
f78: 00 00     DEC  P0
f7a: 00 00     DEC  P0
f7c: 00 00     DEC  P0
f7e: 00 00     DEC  P0
f80: 00 00     DEC  P0
f82: 00 00     DEC  P0
f84: 00 00     DEC  P0
f86: 00 00     DEC  P0
f88: 00 00     DEC  P0
f8a: 00 00     DEC  P0
f8c: 00 00     DEC  P0
f8e: 00 00     DEC  P0
f90: 00 00     DEC  P0
f92: 00 00     DEC  P0
f94: 00 00     DEC  P0
f96: 00 00     DEC  P0
f98: 00 00     DEC  P0
f9a: 00 00     DEC  P0
f9c: 00 00     DEC  P0
f9e: 00 00     DEC  P0
fa0: 00 00     DEC  P0
fa2: 00 00     DEC  P0
fa4: 00 00     DEC  P0
fa6: 00 00     DEC  P0
fa8: 00 00     DEC  P0
faa: 00 00     DEC  P0
fac: 00 00     DEC  P0
fae: 00 00     DEC  P0
fb0: 00 00     DEC  P0
fb2: 00 00     DEC  P0
fb4: 00 00     DEC  P0
fb6: 00 00     DEC  P0
fb8: 00 00     DEC  P0
fba: 00 00     DEC  P0
fbc: 00 00     DEC  P0
fbe: 00 00     DEC  P0
fc0: 00 00     DEC  P0
fc2: 00 00     DEC  P0
fc4: 00 00     DEC  P0
fc6: 00 00     DEC  P0
fc8: 00 00     DEC  P0
fca: 00 00     DEC  P0
fcc: 00 00     DEC  P0
fce: 00 00     DEC  P0
fd0: 00 00     DEC  P0
fd2: 00 00     DEC  P0
fd4: 00 00     DEC  P0
fd6: 00 00     DEC  P0
fd8: 00 00     DEC  P0
fda: 00 00     DEC  P0
fdc: 00 00     DEC  P0
fde: 00 00     DEC  P0
fe0: 00 00     DEC  P0
fe2: 00 00     DEC  P0
fe4: 00 00     DEC  P0
fe6: 00 00     DEC  P0
fe8: 00 00     DEC  P0
fea: 00 00     DEC  P0
fec: 00 00     DEC  P0
fee: 00 00     DEC  P0
ff0: 00 00     DEC  P0
ff2: 00 00     DEC  P0
ff4: 00 00     DEC  P0
ff6: 00 00     DEC  P0
ff8: 00 00     DEC  P0
ffa: 00 00     DEC  P0
ffc: 00 00     DEC  P0
ffe: 00 00     DEC  P0
